:020000040800F2
:10000000709000209D010008310D00089D0A000835
:100010002D0D000895030008F511000800000000F0
:10002000000000000000000000000000910E000829
:100030004D05000800000000410D0008B501000852
:10004000B7010008B7010008B7010008B7010008B0
:10005000B7010008B7010008B7010008B7010008A0
:10006000B7010008B7010008B7010008B701000890
:10007000B7010008B7010008B7010008B701000880
:10008000B7010008B7010008B7010008B701000870
:10009000B7010008B7010008B7010008B701000860
:1000A000B7010008B7010008B7010008B701000850
:1000B000B7010008B7010008B7010008B701000840
:1000C000B7010008B7010008B7010008B701000830
:1000D000B7010008B7010008B7010008B701000820
:1000E000B7010008B7010008B7010008B701000810
:1000F000B7010008B7010008B7010008B701000800
:10010000B7010008B7010008B7010008B7010008EF
:10011000B7010008B7010008B7010008B7010008DF
:10012000B7010008B7010008B7010008B7010008CF
:10013000B7010008B7010008B7010008B7010008BF
:10014000B7010008B7010008B7010008B7010008AF
:10015000B7010008B7010008B7010008B70100089F
:10016000B7010008B7010008B7010008B70100088F
:10017000B7010008B7010008B7010008B70100087F
:10018000B7010008B7010008DFF80CD000F064F8F0
:10019000004800474D1C000870900020064880472A
:1001A00006480047FEE7FEE7FEE7FEE7FEE7FEE75C
:1001B000FEE7FEE7FEE7FEE7ED1000088901000814
:1001C000421C10F8011B0029FBD1801A704770B542
:1001D000064601F06DFC046805460A2200213046FF
:1001E00000F002F82C6070BD2DE9F04791460F46F3
:1001F00080460446002614F8015B2DB100F03EF85D
:100200000068405DC007F6D12B2D02D02D2D18D0EF
:10021000641E4A463946204600F034F827B1396852
:10022000A14201D1C7F8008071054FF002040BD53F
:100230004042002803DD01F03BFC0460A007BDE85C
:10024000F08746F48066E4E70028F8DA01F030FC35
:1002500004606FF00040F2E7064C074D06E0E068EE
:1002600040F0010394E8070098471034AC42F6D3FD
:10027000FFF78EFF6058000880580008004870475C
:10028000C05700082DE9F05F824600780027154628
:100290008B460AF10104B946302801D09DB113E024
:1002A00014F8010B0127782803D0582801D045B154
:1002B0000AE00DB1102D07D10027102514F8010B0D
:1002C00002E0082500E00A250026B0460EE005FB06
:1002D000080005FB06F1012701EB10461FFA80F824
:1002E000B6F5803F00D3B94614F8010B294600F05B
:1002F00018F80028EBDABBF1000F05D00FB1641E2F
:1003000000E05446CBF80040B9F1000F06D001F0F0
:10031000CFFB02210160C81EBDE8F09F48EA0640FD
:10032000FAE73A2800D2303820F02002412A01D3DF
:10033000A2F13700884201D34FF0FF30704770B50B
:100340008C1810F8015B15F0070301D110F8013B80
:100350002A1106D110F8012B03E010F8016B01F807
:10036000016B5B1EF9D12B0705D40023521E0DD45F
:1003700001F8013BFAE710F8013BCB1A921C03E0AD
:1003800013F8015B01F8015B521EF9D5A142D8D3E5
:10039000002070BD00BFFEE70146302905DB39298A
:1003A00003DCA1F13000C0B27047612905DB66298A
:1003B00003DCA1F15700C0B2F6E7412905DB46296D
:1003C00003DCA1F13700C0B2EEE73720ECE7000014
:1003D00010B5394800683949884208D23648001DAE
:1003E00037490860001F00683649086001E000F0E6
:1003F000EBFD35A000F04EFD002858D035480068D0
:1004000000785B2804D133480068401C31490860FB
:10041000002404E000F0D6FA2F490855641C042C8F
:10042000F8DB2EA000F036FDA8B12A48006800785D
:100430005B2804D127480068401C26490860002436
:1004400006E000F0BFFAC1B2234808300155641C31
:10045000042CF6DB08E0FF201F490872FF211E482C
:10046000417200218172C1721FA000F013FDA8B17A
:100470001848006800785B2804D116480068401CC2
:1004800014490860002406E000F09CFAC1B212484A
:10049000001D0155641C042CF6DB0BE000200E4906
:1004A000087100210C4841718171C17102E000F0B6
:1004B0008BFD10BD00BFFCE700000E08C0D401009A
:1004C000D0000020C4000020435F49505F414444F5
:1004D00052000000EC000020E4020020435F49507D
:1004E0005F4D41534B000000435F49505F4741540B
:1004F0004500000010B500220268134B1A40CC687A
:100500000B6823434C6923438C692343CC69234301
:100510000C6A23434C6A23438C6A23434C6B23436A
:100520008C6B23431A430260426922F00702D1E92F
:100530000B3423431A4342610B6943604B68836069
:100540008B68C36010BD00003F801CF07047000046
:1005500001490860704700000C3C024070B5044639
:100560000A460026082502B909E0012A01D116022F
:1005700005E0022A01D1160201E04FF4407600F0B6
:1005800097F80546082D28D11548006820F44070DA
:100590001349086008460068304308600846006850
:1005A00020F0F80008600846006844F002010843A3
:1005B0000B4908600846006840F48030086000F08D
:1005C00077F805460648006820F0020004490860F4
:1005D0000846006820F0F8000860284670BD00005A
:1005E000103C024008201049096801F48031B1F53F
:1005F000803F01D1012015E00B49096801F010018D
:1006000009B105200EE00849096801F0EF0109B1C0
:10061000062007E00449096801F0020109B107203A
:1006200000E00820704700000C3C024003480068CE
:1006300040F000400149086070470000103C024053
:1006400030B502460C46082500F032F80546082D64
:1006500017D10D48006820F440700B490860084627
:10066000006808600846006840F0010008601470E7
:1006700000F01EF805460448006820F00100024919
:100680000860284630BD0000103C02400548006864
:1006900000F0004028B1044802490C3908600348C2
:1006A00008607047103C024023016745AB89EFCDDD
:1006B00008B508200090FFF795FF009002E0FFF7D3
:1006C00091FF00909DF800000128F8D09DF80000EF
:1006D00008BD000010B50446FFF7D8FFF320FFF770
:1006E00037FF02211820FFF739FF00201B4908605F
:1006F00025E01A480068205C7D2800D123E01748D7
:100700000068205C202800D11DE014480068205CAF
:100710000A2800D117E011480068205C0D2800D19C
:1007200011E00E4A1268A15C0C4A12680C4BD018FA
:10073000FFF786FF09480068401C08490860074821
:100740000068FF28D5D900BF04490968044A881801
:100750000021FFF775FFFFF769FF10BD9000002033
:1007600000C0000810B50446FFF790FFF320FFF724
:10077000EFFE00204549086080E045480068454993
:10078000884207D102212020FFF7E8FE082801D087
:1007900000BFFEE73E4800683F49884207D102217A
:1007A0002820FFF7DBFE082801D000BFFEE738480D
:1007B00000683A49884207D102213020FFF7CEFE77
:1007C000082801D000BFFEE731480068344988425C
:1007D00007D102213820FFF7C1FE082801D000BF51
:1007E000FEE72B4800682F49884207D102214020AC
:1007F000FFF7B4FE082801D000BFFEE724480068D8
:100800002949884207D102214820FFF7A7FE08287E
:1008100001D000BFFEE71E4800682449884207D186
:1008200002215020FFF79AFE082801D000BFFEE702
:10083000174800681749884216D3154800681C49B4
:10084000884211D21B4811490968405CFF280BD02F
:1008500018480E4A1268815C0D480068FFF7F0FEE8
:10086000082801D000BFFEE709480068401C08497D
:10087000086006480068401C044908600348006896
:10088000A042FFF47AAFFFF7D1FE10BD9000002028
:10089000E800002000000108000002080000040831
:1008A000000006080000080800000A0800000C0804
:1008B00000000E0843830020F0B50A460021002303
:1008C000002400BF3DE0012505FA01F3156805EAA3
:1008D00003049C4234D105684F000326BE40B54353
:1008E000056015794E00B5400668354305601579F9
:1008F000012D02D01579022D16D185684F000326EF
:10090000BE40B543856055794E00B5408668354395
:100910008560456801268E40B543456045689679F7
:100920008E40B6B235434560C5684F000326BE40D1
:10093000B543C560D5794E00B540C6683543C5603E
:10094000491C1029BFD3F0BDF0B5002300244D078A
:10095000ED0E02FA05F3CE1000F1200555F82650F1
:100960004E07F70E0F26BE40B543CF1000F120060C
:1009700046F82750CE1000F1200555F8265045EADC
:100980000304CE1000F1200545F82640F0BD418358
:1009900070470183704730B5024612F8010BFFF72C
:1009A000FBFC0446102C01DD002030BD1078FFF761
:1009B000F3FC0346102B01DD0020F6E703EB0410E7
:1009C000C0B2F2E710B50C48006800785D2801D18C
:1009D000002010BD08480068FFF7F9FB84B200BF93
:1009E00005480068017804480068401C024A10600D
:1009F0002C29F5D12046ECE7EC00002070B502254B
:100A00002248234908600846006800783A281BD12C
:100A100015E01F480068007853280BD11C48006877
:100A2000401C1B49086008460068FFF7D0FB0546DC
:100A3000284670BD16480068401C154908601448D7
:100A4000006800780028E4D11248114908600024A9
:100A500016E00F480068006800B90BE00C48006819
:100A600000680D49884200D90CE009480068056813
:100A70002846DEE7641C06480068001D044908603B
:100A8000082CE6D300BF2846D3E7000000C00008CA
:100A9000900000200078FF1F9999990000BFFEE7A1
:100AA00001464FF48042224B1A800A0A214B1A73E6
:100AB00000BF204A127A02F00102002AF9D01D4A32
:100AC000127B1C4B197300BF1A4A127A02F0010202
:100AD000002AF9D0174A127B0022164B1A7300BF66
:100AE000144A127A02F00102002AF9D0114A127B4C
:100AF0000122104B1A7300BF0E4A127A02F0010253
:100B0000002AF9D00B4A127B00220A4B1A7300BF4D
:100B1000084A127A02F00102002AF9D0054A107B35
:100B200000BF4FF48042024B9B1E1A8070470000AA
:100B30001A0C02400030014010B501464FF48040CD
:100B4000284B1880080A284B187300BF2648007AE3
:100B500000F001000028F9D02348007B224B1973D4
:100B600000BF2148007A00F001000028F9D01E489B
:100B7000007B00201C4B187300BF1B48007A00F05C
:100B800001000028F9D01848007B0220164B18738A
:100B900000BF1548007A00F001000028F9D0124883
:100BA000007B0020104B187300BF0F48007A00F044
:100BB00001000028F9D00C4B187B020200201873AA
:100BC00000BF0948007A00F001000028F9D0064B68
:100BD000187B02434FF48043024CA41E238010462E
:100BE00010BD00001A0C02400030014002464FF4D4
:100BF0008040214B1880100A204B187300BF1F48FB
:100C0000007A00F001000028F9D01C48007B1B4B43
:100C10001A7300BF1948007A00F001000028F9D0CB
:100C20001648007B8020154B187300BF1348007ACC
:100C300000F001000028F9D01048007B01200F4B84
:100C4000187300BF0D48007A00F001000028F9D0A9
:100C50000A48007B0948017300BF0848007A00F089
:100C600001000028F9D00548007B4FF48040024B7A
:100C70009B1E1880012070471A0C02400030014072
:100C800002464FF48040274B1880100A264B1873F9
:100C900000BF2548007A00F001000028F9D0224862
:100CA000007B214B1A7300BF1F48007A00F001003F
:100CB0000028F9D01C48007B80201B4B187300BF14
:100CC0001948007A00F001000028F9D01648007B8E
:100CD0000220154B187300BF1348007A00F0010082
:100CE0000028F9D01048007B080A0F4B187300BF8A
:100CF0000D48007A00F001000028F9D00A48007B76
:100D0000094B197300BF0848007A00F00100002861
:100D1000F9D00548007B4FF48040024B9B1E1880A1
:100D2000012070471A0C02400030014000BFFEE76E
:100D300070470000014908627047000000000E4241
:100D40007047000029B1064A12680243044B1A603A
:100D500004E0034A12688243014B1A6070470000A6
:100D60003038024029B1064A12680243044B1A6027
:100D700004E0034A12688243014B1A607047000086
:100D80004038024029B1064A12680243044B1A60F7
:100D900004E0034A12688243014B1A607047000066
:100DA0002038024029B1064A12680243044B1A60F7
:100DB00004E0034A12688243014B1A607047000046
:100DC0004438024029B1064A12680243044B1A60B3
:100DD00004E0034A12688243014B1A607047000026
:100DE0002438024021B1028842F04002028004E02F
:100DF00002884FF6BF731A400280704710B5044650
:100E00001148844208D101218014FFF7DBFF002143
:100E1000A014FFF7D7FF16E00C48844208D1012147
:100E20000014FFF7AFFF00212014FFF7ABFF0AE02B
:100E30000748844207D10121C013FFF7A3FF002117
:100E4000E013FFF79FFF10BD003001400038004065
:100E5000003C004010B50022028802F441520B8889
:100E60004C8823438C882343CC8823430C89234319
:100E70004C8923438C892343CC8923431A43028022
:100E8000838B4FF2FF74234083830B8A038210BD50
:100E90007047000002462A4800682A4B18604AE062
:100EA00028480068007800B946E0264800680078C5
:100EB000FF2800D140E02348006800787D2800D159
:100EC0003AE0204800680078222805D01D480068D4
:100ED000401C1C4B18602EE01A480068401C194B3F
:100EE0001860184600680078137898421DD10021D8
:100EF00008E0505C134B1B685B5C984200D004E038
:100F0000481CC1B2505C0028F3D100BF505C60B9EE
:100F10000C480068405C222807D10A480368C81CB6
:100F20001844084B18600120704706480068401CB0
:100F3000044B186000BFB3E700BF0020F4E70000D7
:100F4000D0000020EC00002010B503461D480360CF
:100F500033E01C480068007800B92FE019480068A9
:100F60000078FF2800D129E01648006800787D2825
:100F700000D123E01348006800780C78A04217D114
:100F800000220DE0885C0F4C24682478A04200D039
:100F900009E00C480068401C0A4C2060501CC2B29A
:100FA000885C0028EED100BF885C08B9012010BD24
:100FB00004480068401C034C2060CAE700BF0020C2
:100FC000F5E70000EC000020C0200C490870A820C4
:100FD0004870012088700220C870FF200872FF212D
:100FE0000648417200218172C172002003490871D4
:100FF0000021024841718171C1717047E4020020F3
:101000000CB50020019000903448006840F4803016
:101010003249086000BF3148006800F40030009099
:101020000198401C0190009818B90198B0F5A04FA4
:10103000F1D12A48006800F4003010B1012000907E
:1010400001E0002000900098012846D1234840305C
:10105000006840F080502149403108602048006815
:1010600040F440401E4908601C48083000681B4995
:10107000083108600846006840F4204008600846CF
:10108000006840F4A05008601648091F0860081F57
:10109000006840F08070091F086000BF0F480068BA
:1010A00000F000700028F9D040F205600E49086099
:1010B0000A480830006820F0030008490831086039
:1010C0000846006840F00200086000BF034808308E
:1010D000006800F00C000828F8D10CBD0038024070
:1010E0000070004019544007003C024010B51648FB
:1010F000006840F0010014490860002012490831DE
:10110000086011480068114908400F4908601048FC
:10111000091D0860081F006820F48020091F08606E
:10112000002009490C310860FFF76AFF4FF00060AA
:101130000849086007488030006840F4700005499D
:101140008031086010BD000000380240FFFFF6FE4D
:101150001030002408ED00E021B1028842F00102C5
:10116000028004E002884FF6FE731A400280704746
:1011700000220288184B98420ED0184B98420BD090
:10118000B0F1804F08D0164B984205D0154B9842CD
:1011900002D0154B984204D14FF68F731A404B88FA
:1011A0001A43124B984207D0114B984204D04FF685
:1011B000FF431A400B891A4302804B68C3620B88B5
:1011C0000385054B984202D0044B984201D18B7A9B
:1011D0000386012383827047000001400004014020
:1011E0000004004000080040000C004000100040D7
:1011F0000014004000BFFEE730B503461D480168FB
:101200001D4800881D4C246860830020087100BFC1
:10121000087800F001000028FAD008790B7100BFAF
:10122000087800F001000028FAD008790020087141
:1012300000BF087800F001000028FAD008790020EB
:10124000087100BF087800F001000028FAD0087982
:1012500002020020087100BF087800F00100002899
:10126000FAD008790243044C2488044D2D682C835D
:10127000104630BDB4010020B8010020B0010020AC
:1012800030B502460B461A4C2168012404EB820457
:10129000E200184C2488184D2D686C8300240C71D2
:1012A00000BF0C7804F00104002CFAD00C790B710B
:1012B00000BF0C7804F00104002CFAD00C790A71FC
:1012C00000BF0C7804F00104002CFAD00C79002443
:1012D0000C7100BF0C7804F00104002CFAD00879DE
:1012E00000BF044C2488044D2D682C8330BD0000C1
:1012F000B4010020B8010020B001002070B5024602
:101300000C461F480168012000EB8200C2001D4806
:1013100000881D4D2D6868830020087100BF087883
:1013200000F001000028FAD008790C7100BF08789D
:1013300000F001000028FAD008790A7100BF08788F
:1013400000F001000028FAD008790020087100BFE1
:10135000087800F001000028FAD008790302002084
:10136000087100BF087800F001000028FAD0087961
:101370000343044D2D88044E36683583184670BDEE
:10138000B4010020B8010020B001002030B50246B1
:101390000B461748016817480088174C246860837B
:1013A0000020087100BF087800F001000028FAD082
:1013B00008790A7100BF087800F001000028FAD00F
:1013C00008790420087100BF087800F001000028A7
:1013D000FAD008790B7100BF087800F001000028EE
:1013E000FAD00879034C2488034D2D682C8330BD36
:1013F000B4010020B8010020B001002030B5034640
:101400000A461C4801681C4800881C4C24686083FC
:101410000020087100BF087800F001000028FAD011
:1014200008790B7100BF087800F001000028FAD09D
:1014300008790420087100BF087800F00100002836
:10144000FAD00879100A087100BF087800F001008E
:101450000028FAD008790A7100BF087800F001006E
:101460000028FAD00879044C2488044D2D682C8378
:1014700030BD0000B4010020B8010020B001002000
:1014800070B503460C4619480168012000EB830043
:10149000C30017480088174D2D6868830020087125
:1014A00000BF087800F001000028FAD008790C711C
:1014B00000BF087800F001000028FAD00879181D54
:1014C000087100BF087800F001000028FAD0087900
:1014D0000A7100BF087800F001000028FAD00879EE
:1014E000034D2D88034E3668358370BDB40100204E
:1014F000B8010020B001002070B503460C461E481C
:101500000168012000EB8300C3001C4800881C4DCB
:101510002D6868830020087100BF087800F0010082
:101520000028FAD008790C7100BF087800F001009B
:101530000028FAD00879181D087100BF087800F05B
:1015400001000028FAD00879100A087100BF087855
:1015500000F001000028FAD008790A7100BF08786D
:1015600000F001000028FAD00879044D2D88044EBF
:101570003668358370BD0000B4010020B80100203A
:10158000B00100200549064A11604FF48041054A28
:1015900011600549054A116070470000000C0240C7
:1015A000B0010020B801002008300140B401002043
:1015B00010B5052203216248FFF7C6F90522042170
:1015C0005F48FFF7C1F9052211465D48FFF7BCF9F6
:1015D00002205C490871002088710220C87148719E
:1015E000082008605648FFF767F920205549086031
:1015F0005348FFF761F91020524908605048FFF73F
:101600005BF95148FFF7FAFB0020504908808880B9
:10161000C88008814FF40070488100208881C8810B
:10162000072008824FF4827048804748FFF712FC79
:1016300001214548FFF7D6FB0420424908600120FC
:10164000087100208871022048714148FFF734F981
:1016500004213F48FFF79BF94FF4404039490860A7
:101660000120087100208871022048713948FFF775
:1016700023F94FF440413748FFF78BF901203149F6
:101680000860087100208871022048713048FFF717
:1016900013F901212E48FFF77AF900202949087132
:1016A000C8714FF4006008602B48FFF705F94FF050
:1016B000C0602A49086024480C3048602848886087
:1016C0000020C86093200861002048614FF48060CA
:1016D00088610020C861086248624FF40030886267
:1016E0000020C862012008630020486388631D4809
:1016F000FEF700FF4FF0C0601849086012480C3038
:101700004860194888604020C86093200861002024
:1017100048614FF4806088610020C86108624862B7
:101720004FF4003088620020C86201200863002066
:10173000486388630B481830FEF7DCFE10BD0000DC
:1017400000040240640000200030014068020020D4
:1017500000180240000C0240001402407C020020ED
:10176000438B0020406402400001002010B5052298
:1017700003215A48FFF7E8F8052204215748FFF7EC
:10178000E3F8052211465548FFF7DEF802205449D8
:101790000871002088710220C87148710820086013
:1017A0004E48FFF789F820204D4908604B48FFF765
:1017B00083F810204A4908604848FFF77DF84948F7
:1017C000FFF71CFB0020484908808880C8800881FA
:1017D0004FF40070488100208881C881072008826A
:1017E0004FF4827048803F48FFF734FB01213D48A9
:1017F000FFF7F8FA4FF440403949086001200871BA
:1018000000208871022048713848FFF755F84FF4DE
:1018100040413648FFF7BDF80120314908600871A2
:1018200000208871022048713148FFF745F80121F6
:101830002F48FFF7ACF8002029490871C8714FF410
:10184000006008602B48FFF737F84FF0C0602A4966
:10185000086024480C304860284888600020C86030
:1018600079200861002048614FF480608861002081
:10187000C861086248624FF4003088620020C86284
:10188000012008630020486388631D48FEF732FE8C
:101890004FF0C0601849086012480C304860194881
:1018A00088604020C86079200861002048614FF4BA
:1018B000806088610020C861086248624FF400308F
:1018C00088620020C86201200863002048638863A2
:1018D0000B481830FEF70EFE10BD00000004024059
:1018E000640000200030014068020020000C02402B
:1018F00000180240001402407C020020438B0020AC
:1019000040640240BC01002000B50920FFF714F933
:1019100000BD00B50920FFF76FFC00BD10B50446FF
:101920004FF4804101EB0421491C8AB20221104688
:10193000FFF75CF900BF4FF4804202EB0422521C17
:1019400091B20846FFF7ACF80028F4D110BD10B5ED
:101950000446022201212046FFF792FD00BF01212B
:101960002046FFF78DFC0028F9D110BDF0B50446E4
:101970000F4615461E464FF4804101EB04218AB202
:1019800039461046FFF732F94FF4804101EB04214C
:10199000091D8AB229461046FFF772F94FF48041BB
:1019A00001EB042110318AB231461046FFF768F985
:1019B0004FF4804101EB0421491C8AB201211046F9
:1019C000FFF714F900BF4FF4804202EB0422521CCF
:1019D00091B20846FFF764F80028F4D1F0BDF0B5E5
:1019E00006460C4617461D46224600213046FFF7A4
:1019F00047FD3A4604213046FFF77EFD2A46102176
:101A00003046FFF779FD012211463046FFF738FDD9
:101A100000BF01213046FFF733FC0028F9D1F0BDAB
:101A200010B5044621780920FFF7E0F861780A2014
:101A3000FFF7DCF8A1780B20FFF7D8F8E1780C204D
:101A4000FFF7D4F821790D20FFF7D0F861790E2047
:101A5000FFF7CCF810BD10B5044621780920FFF738
:101A600095FC61780A20FFF791FCA1780B20FFF725
:101A70008DFCE1780C20FFF789FC21790D20FFF720
:101A800085FC61790E20FFF781FC10BD0FB408467C
:101A900010B5064A02A900F01EF8044602A900206B
:101AA00000F02AF8204610BC5DF814FBF91A000873
:101AB000004870473C02002002E008C8121F08C11D
:101AC000002AFAD170477047002001E001C1121FBF
:101AD000002AFBD170472DE9F04116460F46044617
:101AE000002503E03946B047641C6D1C20780028AF
:101AF000F8D12846BDE8F0810A68531C0B601070CD
:101B0000704710B504464FF4804101EB0421491C95
:101B10008AB210211046FFF769F800BF4FF48042E7
:101B200002EB0422521C91B20846FEF7B9FF0028CE
:101B3000F4D14FF4804101EB0421891C8AB2FF21CA
:101B40001046FFF753F810BD10B5044610220121CE
:101B50002046FFF795FC00BF01212046FFF790FBD0
:101B60000028F9D1FF2202212046FFF789FC10BD91
:101B700010B504464FF4804101EB0421491C8AB2A0
:101B800008211046FFF732F800BF4FF4804202EB05
:101B90000422521C91B20846FEF782FF0028F4D1BD
:101BA00010BD10B50446082201212046FFF768FC4D
:101BB00000BF01212046FFF763FB0028F9D110BDCB
:101BC0000146CA0202F5404290B270470146CA027D
:101BD00002F5004290B2704710B504464FF48042BF
:101BE00002EB0422263291B20846FEF7A5FF10BD93
:101BF00010B5044626212046FFF780FB10BD10B526
:101C000004464FF4804202EB0422D21C91B20846F3
:101C1000FEF746FF10BD10B5044603212046FFF72E
:101C20002FFB10BD10B504464FF4804202EB042296
:101C3000203291B20846FEF77FFF10BD10B5044672
:101C400020212046FFF75AFB10BD0000FE488068A7
:101C500040F48050FC4988600121FC48FFF772F88D
:101C6000012141F21000FFF79DF80121F848FFF72C
:101C700079F80120FFF75EF8F648006840F48070BC
:101C8000F44908600020F44908710120C8717F20E0
:101C90000860F248FEF710FEF14C282503E0641EB0
:101CA0000CB96D1EEE4CED48006900F0100008B94B
:101CB000002DF4DC35B90020EA4988600120EA49AA
:101CC000088067E00020E8490880E6488068E74926
:101CD000884212D10020E34988604CF6CC40E449A8
:101CE000086045F255500860012048601020886067
:101CF0004AF6AA20086000BFFEE7DA488068DD499E
:101D0000884246D0DC480068DC490840B0F1005FFA
:101D10003FD1D948006ADA490860D748406AD949B2
:101D20000860D5483030D8490860D5480068B0F51B
:101D3000503F00D92EE0D3480068D0B10120D349EC
:101D4000886000240AE0D04800680068CF49086035
:101D5000CD480068001DCC490860641CC848006874
:101D60008442F0D3C9480068C6490968884200D057
:101D700010E0C1484068C649086008460068C54987
:101D80000860BD49086880F3088800BFC148006842
:101D9000804700BF0220B0490871002088710220EE
:101DA000C87148714FF4E0500860BB48FEF784FDED
:101DB00006220A21B848FEF7C7FD06220B21B648C5
:101DC000FEF7C2FD06220C21B348FEF7BDFD4FF41D
:101DD0004050A1490860012008710020887102204C
:101DE0004871AE48FEF768FDAD48FFF707F80020E0
:101DF000AC4908808880C88008814FF40070488111
:101E0000282088810020C881072008824FF4827032
:101E10004880A348FFF71EF80121A148FEF7E2FF22
:101E20001420A14908702820487050208870A120F3
:101E3000C87042200871852048710A2088711420DA
:101E4000C8712820087250204872A1208872422050
:101E5000C872852008730A2048734FF480518F4858
:101E6000FEF795FD4FF400518C48FEF790FD8C482D
:101E70000C3000888D490860002089490C310880A9
:101E800000BF87480830008800F001000028F8D023
:101E900083480C300088854908604FF400517F4822
:101EA000FEF777FD002405E07D48083000887F4973
:101EB0000860641CB4F5FA7FF6DB4FF400517748F4
:101EC000FEF765FD4FF480517448FEF762FD002572
:101ED0002CE073480C300088744908607248405DFB
:101EE0006F490C31088000BF6D480830008800F051
:101EF00001000028F8D06A480C3000886B4908605F
:101F00004FF400516548FEF744FD002405E06448A5
:101F10000830008865490860641CB4F5FA7FF6DB78
:101F20004FF400515D48FEF732FD6D1C0E2DD0DBE5
:101F30004FF480515948FEF72AFD00215848FEF71A
:101F400051FF5748FEF75AFF0020564908804FF4CA
:101F5000006088800020C88008814FF400704881AC
:101F6000282088810020C881072008824FF48270D1
:101F700048804B48FEF76EFF01214948FEF732FFCB
:101F80000020354908710120C8717F20086033485E
:101F9000FEF792FC314801697F20884320F0100051
:101FA000434908600020434908604148007800F038
:101FB0000100002846D04048404908604048414957
:101FC0000860414841490860414842490860424828
:101FD0004249086042484349086043484349086011
:101FE00043484449086044484449086044484549D6
:101FF00008604548454908604548464908604648E4
:1020000046490860464847490860474847490860CC
:10201000474848490860484848490860484849498D
:1020200008604948494908602248006840F48040F7
:1020300020490860FFF7A6FA1E48006840F4805067
:102040001C4985E086E00000002004E07F10640069
:102050000180001000700040640000200010024069
:1020600040420F00004002408E000020009125FCFD
:102070000030004071554812000001080000FE2F9A
:1020800080000020840000208800002000300240F2
:10209000F4000020F000002000080240000C024084
:1020A000003C004068020020438300209000002094
:1020B000F8000020FC000020A31B000818000020EE
:1020C0005D2D00081C0000203D320008200000208B
:1020D000C92F000824000020491B00082800002008
:1020E000DF1900082C0000204F19000830000020E4
:1020F000F11B0008340000206B3400083800002079
:10210000571A00083C00002023330008400000203C
:102110000F34000844000020573300084800002016
:102120008F3300084C00002073330008500000205B
:102130001319000854000020C33300085800002081
:102140003D1C00085C000020171C000860000020F7
:10215000086040E0F348F4490860F448F449086036
:10216000F448F5490860F548F5490860F548F6492E
:102170000860F648F6490860F648F7490860F748ED
:10218000F7490860F748F8490860F848F8490860D6
:10219000F848F9490860F948F9490860F948FA49E6
:1021A0000860FA48FA490860FA48FB490860FB48A9
:1021B000FB490860FB48FC490860FC48FC49086092
:1021C000FC48FD490860FD48006840F48050FB4928
:1021D0000860FFF7D7F9FA48008810B1FEF7F4FE5F
:1021E00001E0FEF7F5F8F7488068F74988420CD11E
:1021F000F448C06848B1F348C068F4490860F14841
:1022000040698860EF48006948600020ED498860B7
:10221000FEF7F4FBEE490860EE4800684008EE491E
:10222000B0FBF1F0401EED49088000204880401EC0
:1022300048600020088188724FF08040FEF798FFC8
:1022400001218807FEF788FFDC48008800F4804001
:1022500010B1FFF78BFA01E0FFF7AAF90121E0487E
:10226000FEF795FB00204FF0804148620846406A27
:10227000DC490844DC49086000BF4FF08040406AF8
:10228000D94909688842F8D30121D548FEF781FB76
:1022900000204FF0804148620846406AD349084414
:1022A000D149086000BF4FF08040406ACE490968BC
:1022B0008842F8D30020CE490860C5480068CA4962
:1022C00008600846006842F21071B0FBF1F00404A7
:1022D000C5480068B0FBF1F201FB1200C24908607A
:1022E000084600684FF47A71B0FBF1F004EB00345B
:1022F000BD480068B0FBF1F201FB1200BA4908606A
:10230000084600686421B0FBF1F004EB0024B648F5
:102310000068B0FBF1F201FB1200B3490860084607
:1023200000680A21B0FBF1F004EB0014AE4800682D
:10233000B0FBF1F201FB1200AB49086008460068EF
:1023400020440860FA20AB490870CE204870102065
:102350008870A5480068000CC870A3480088000A6F
:102360000871A14800784871084681490968884782
:1023700096488D490968884794480830804909681B
:1023800088479248001D7C49096888474FF47A6065
:102390007F490968884703207F4909688847724850
:1023A000006880474CF6CC409349086045F2555090
:1023B0000860042048604FF47A7088604AF6AA20CA
:1023C000086000204FF0804148620846406A854915
:1023D00008448A490860002089490860ECE34AF60D
:1023E000AA20854908604007406A844909688842F4
:1023F0007ED900204FF0804148620846406A794902
:1024000008447E4908607E480068401C7C4908609A
:102410000846006840F6B83188420FD94CF6CC40E7
:102420007549086045F25550086001204860102049
:1024300088604AF6AA20086000BFFEE7714800687D
:10244000401C704908600846007800F0040008B39A
:102450004FF400516C48FEF79AFA6C4800886249C4
:10246000086045F255506949088000BF6748001F61
:10247000008800F001000028F8D0644800885A491C
:1024800008604FF400516048FEF783FA00205D4970
:10249000086024E04FF400515B48FEF778FA5B488F
:1024A0000088514908605A48008820B14AF6AA209D
:1024B0005649088002E000205449088000BF534874
:1024C000001F008800F001000028F8D04F48008865
:1024D000454908604FF400514B48FEF75AFA4C4802
:1024E0000088B0F57A7F03DD49480088401E00E08F
:1024F00016E04749088008460088B0F57A7F0FDC6F
:102500004CF6CC403C49086045F25550086001202B
:102510004860102088604AF6AA20086000BFFEE7E5
:1025200078E00000711B000818000020132D00083F
:102530001C000020FB310008200000206D2E000848
:1025400024000020031B0008280000206D1900084B
:102550002C0000201D19000830000020D91B0008A5
:10256000340000203534000838000020211A00080B
:102570003C000020FD32000840000020E933000844
:10258000440000204933000848000020813300083F
:102590004C00002065330008500000200919000895
:1025A000540000209D33000858000020251C00081E
:1025B0005C000020FF1B000860000020FC000020E1
:1025C0008E0000200040024071554812E4020020B5
:1025D000780000200000002040420F004002002050
:1025E00000180240A08601009000002020A10700F2
:1025F000D8000020DC0000200030004094000020C3
:10260000980000209C000020000C02400C3C004080
:102610008C000020F848006800287DD0F64800684B
:10262000C01E062877D2DFE800F0EAE976A5E803C5
:10263000F2A1F548FEF788FCF0B3FEF727F8F32087
:10264000FDF786FF02215820FDF788FFFDF7EEFF1A
:10265000EE49EF48FFF71AFAED48FDF7B1FDED49F5
:1026600008600846008882B2E9490720EA4B1B68E7
:10267000984700204FF08041486200BF4FF08040F3
:10268000406A4CF250318842F8D30720E349096888
:10269000884700204FF08041486200BF4FF08040E3
:1026A000406A4CF250318842F8D30020DC498860FF
:1026B0004CF6CC40DB4900E00CE0086045F2555098
:1026C000086001204860102088604AF6AA2008604F
:1026D00000BFFEE7D4A1CC48FEF736FCE8B1FDF719
:1026E000D5FFF320FDF734FF02214820FDF736FF28
:1026F000FDF79CFFC549C648FFF7C8F9C448FDF778
:102700005FFDC44908600320BB4908600020C94937
:102710000860C9490860C5E1C5E1C8A1BA48FEF72B
:1027200013FCA8B1C8480068FDF7D4FFB749B84802
:10273000FFF7ACF9B648FDF743FDB6490860032042
:10274000AD4908600020BB490860BB490860A9E1A9
:10275000BE484068BE4908600020B6490860BB48D2
:10276000C068BA494968401AAA4908600320A249CA
:10277000086097E1B7480088F0BBB7A1A248FEF710
:10278000E3FB002871D0A149A148FFF77FF9A048D9
:10279000FDF716FDA84908600846008882B29C49EA
:1027A00007209D4B1B68984700204FF080414862EE
:1027B00000BF4FF08040406A4CF250318842F8D35D
:1027C000072096490968884700204FF080414862F9
:1027D00000BF4FF08040406A4CF250318842F8D33D
:1027E00000208F4988604CF6CC408E49086045F245
:1027F00055500860012003E00AE043E046E1D1E0E3
:102800004860102088604AF6AA20086000BFFEE7F2
:102810007D488D49086000241BE08B4800680078E3
:10282000212804D188480068401C874908608648F0
:10283000006800787D2800D10EE083480068FEF72C
:10284000AAF87349085580480068801C7E490860D2
:10285000641CB4F5806FE0DB00BF14B12046FDF7C7
:1028600081FF4FF47F707B4908807E496848FFF7FD
:102870000DF96748FDF7A4FC6F49086004205E4924
:1028800008600FE173480088B8BB77A15E48FEF787
:102890005BFB98B36C48006800783A2803D00520A9
:1028A00055490860FEE068480068401C66490860B9
:1028B00068480088401C6749088063480068FEF744
:1028C0006AF800066B4908605F480068801C5E4932
:1028D000086008460068FEF75EF86649096841EA44
:1028E00000406449086058480068801C56490860E8
:1028F00060480068604908600CE007E0FFE70020DE
:102900004D49086005203C4908604AE03E484E4970
:10291000086000BF002416E04B48006800787D285E
:1029200004D0494800680078212800D10EE04648CC
:102930000068FEF730F83649085543480068801CA7
:1029400041490860641CB4F5806FE5DB00BF14B139
:102950002046FDF707FF3C480068401C3A490860E4
:10296000002046490860012023490860002415E042
:1029700035480068007828B133480068007822495B
:10298000085500E00CE030480068401C2E49086003
:102990003A480068401C39490860641CFA2CE7DB9F
:1029A00000BF7FE036480068B0F5FA7F6DD9224855
:1029B0000068F0B9002414E01E4800681549096851
:1029C00088420CD2224800681A490968405C1049C4
:1029D000085518480068401C1649086000E003E0EC
:1029E000641CB4F5967FE7DB00BF1CB1124804609D
:1029F0004BE04AE046E00000A8000020436C65611F
:102A000072436F6E6600000044030020C457000844
:102A100043830020B8000020200000201800002080
:102A20000040024000300040436C65617243616CBD
:102A300063000000B4000020AC0000205365745017
:102A40003D7B313739360000EC0000202C57000860
:102A5000CC0000208C00002072756E6D61696E3DA7
:102A60007B000000185800084669726D4845583DC3
:102A70007B000000E4000020E8000020A40000200B
:102A8000C800002004207A4908600BE079480068FB
:102A9000B0F5006F05D17848006810B90520744979
:102AA000086000BF00BF072074490968884790B1DB
:102AB000132804D0172829D01C280BD11AE007208E
:102AC0006F490968884700206E4908606E490860B0
:102AD00067490860C9E000235022012107206B4E9E
:102AE0003668B04700206749086067490860604958
:102AF0000860BAE0072066490968884700206149F4
:102B00000860614908605A490860AEE007206149E1
:102B100009688847574908605548006806287CD2EC
:102B2000DFE800F00304A284859600BF07205A491D
:102B3000096888475949086008460068D8B30846BC
:102B40000068642801D9642008605448008882B273
:102B500053484C4B1B68C1180720524B1B689847C1
:102B60004348006830BB4E48007847280FD14C4896
:102B7000407845280BD14A488078542807D14848E6
:102B8000C078202803D108203949086018E044485B
:102B90000078502811D1424840784F280DD1404844
:102BA0008078532809D13E48C078542805D10120A7
:102BB0002F49086004E038E058E005202C490860FF
:102BC0002B480068012819D1002413E02D48006823
:102BD00020443349085C212802D07D2808D103E035
:102BE00007202349086003E006202149086000BF50
:102BF00000BF641C294800688442E7D3214800686C
:102C00002649096808441F490860002024491D4AD4
:102C1000126888541B48006800E025E047F2FD7107
:102C2000884202D90520124908601DE000BF124801
:102C3000006860B11048008882B21B4907201B4B16
:102C40001B68984700200B4908600B4908600BE09F
:102C500007200F490968884700200A4908600A4987
:102C600008600349086000BF00BF00BFFFF7B7BBA3
:102C7000A8000020C8000020AC0000206000002058
:102C800030000020A4000020B00000202C00002014
:102C9000180000205C00002034000020800000208C
:102CA000440300201C00002043830020200000205B
:102CB0002DE9F0478246894616461C46C9F30A08A4
:102CC0005046FEF77DFF00EB080508EB0400B0F569
:102CD000006F16DDC8F500618FB2ABB23A463146DF
:102CE000184600F0C3FB3E44E11B8FB25046FEF78E
:102CF00067FF05462B463A463146184600F0B6FBBC
:102D000005E0ABB222463146184600F0AFFBBDE805
:102D1000F087F0B504460E4615460027002D1BDD52
:102D20002A463146204600F07FF84FF4804101EBFF
:102D30000421491C8AB240211046FDF757FF00BF0D
:102D40004FF4804202EB0422521C91B20846FDF778
:102D5000A7FE0028F4D12F463846F0BD2DE9F043F8
:102D600081460F4615462D490C6828214846FEF736
:102D7000C5FA06462A4800882A490968488330125D
:102D8000207100BF207800F001000028FAD02079DF
:102D9000267100BF207800F001000028FAD02079C9
:102DA0004FEA8900C01C002101EBC000207100BF68
:102DB000207800F001000028FAD020794FF00008B8
:102DC0000EE00020207100BF207800F001000028F4
:102DD000FAD0207938707F1C08F101001FFA80F8C2
:102DE000A845EEDB0E4909880E4A12681183711955
:102DF0008EB2324628214846FEF77EFB4022012152
:102E00004846FEF73DFB00BF01214846FEF738FA71
:102E10000028F9D12846BDE8F0830000B401002065
:102E2000B8010020B0010020F0B504460E4615465A
:102E30004FF4804202EB0422283291B20846FDF79B
:102E40007BFE07462B46324639462046FFF730FFC9
:102E500079198FB24FF4804101EB042128318AB2F5
:102E600039461046FDF70CFFF0BD00002DE9FC438C
:102E700004468946154698464FF4804202EB0422E8
:102E8000283291B20846FDF757FE07464FF48042BC
:102E900002EB042291B20846FDF702FE00F00700A3
:102EA000022804D003282BD0042856D144E008235C
:102EB0006A4639462046FFF7FBFE07F1080087B255
:102EC0009DF8000028709DF8010068709DF80200D0
:102ED000A8709DF80300E8709DF80400A8F80000B1
:102EE0009DF8050098F8001000EB0120A8F80000FC
:102EF0009DF806609DF8070000EB062086B22DE0E5
:102F000006236A4639462046FFF7D2FEB81D87B22F
:102F10009DF8000028709DF8010068709DF802007F
:102F2000A8709DF80300E8709DF804609DF8050006
:102F300000EB062086B211E002236A46394620469D
:102F4000FFF7B6FEB81C87B29DF800609DF801003F
:102F500000EB0620801E86B200E000BF00BFB6F581
:102F6000007F06DA33464A4639462046FFF7A0FE80
:102F700000E00026B9198FB212490F804FF480414A
:102F800001EB042128318AB239461046FDF778FE5C
:102F90004FF4804101EB0421491C8AB240211046C4
:102FA000FDF724FE00BF4FF4804202EB0422521CC6
:102FB00091B20846FDF774FD0028F4D13046BDE813
:102FC000FC830000AC0100202DE9FF4B8146154633
:102FD000984676490C6828214846FEF78FF907463F
:102FE000734800887349096848833812207100BF0C
:102FF000207800F001000028FAD02079277100BF66
:10300000207800F001000028FAD020794FEA8900EA
:10301000C01C002101EBC000207100BF207800F02F
:1030200001000028FAD020790020207100BF20780C
:1030300000F001000028FAD02079287000202071CB
:1030400000BF207800F001000028FAD020796D1C24
:1030500028700020207100BF207800F001000028B7
:10306000FAD020796D1C28700020207100BF2078D4
:1030700000F001000028FAD020796D1C2870002093
:10308000207100BF207800F001000028FAD02079DC
:10309000A8F800000020207100BF207800F0010097
:1030A0000028FAD0207998F8001000EB0120A8F849
:1030B00000000020207100BF207800F001000028EF
:1030C000FAD0207906460020207100BF207800F059
:1030D00001000028FAD0207900EB062086B234489F
:1030E000008834490968088307F1080087B2B6F5FB
:1030F000007F40DC2E4800882E490968488338123A
:10310000207100BF207800F001000028FAD020795B
:10311000277100BF207800F001000028FAD0207944
:103120004FEA8900C01C002101EBC000207100BFE4
:10313000207800F001000028FAD020794FF0000B31
:1031400012E00020207100BF207800F0010000286C
:10315000FAD020792179019801700198401C0190E2
:103160000BF101001FFA80FBB345EADB1048008831
:10317000104909680883B9198FB23A462821484690
:10318000FEF7BAF9402201214846FEF779F900BF5F
:1031900001214846FEF774F80028F9D1B6F5007F02
:1031A00002DD04B0BDE8F08B3046FAE7B401002040
:1031B000B8010020B0010020F0B504460F461546C6
:1031C0004FF4804202EB0422243291B20846FDF70C
:1031D000B3FC06462B4632463946204600F0FAF943
:1031E00071198EB24FF4804101EB042124318AB26F
:1031F00031461046FDF744FDF0BD70B504460D465E
:103200001646324629462046FFF7D6FF4FF4804146
:1032100001EB0421491C8AB220211046FDF7E6FC8F
:1032200000BF4FF4804202EB0422521C91B20846C8
:10323000FDF736FC0028F4D170BD00002DE9F04305
:103240008046894617462A490C6824214046FEF7E5
:1032500055F80546274800882749096848832812F9
:10326000207100BF207800F001000028FAD02079FA
:10327000257100BF207800F001000028FAD02079E5
:103280004FEA8800801C042101EBC000207100BFC0
:10329000207800F001000028FAD0207900260AE00A
:1032A00019F80600207100BF207800F00100002806
:1032B000FAD02079761CBE42F2DB0E4909880E4A0C
:1032C00012681183E9198DB22A4624214046FEF77F
:1032D00013F9202201214046FEF7D2F800BF012158
:1032E0004046FDF7CDFF0028F9D1BDE8F08300008E
:1032F000B4010020B8010020B001002010B5044640
:1033000021780120FDF772FC61780220FDF76EFC48
:10331000A1780320FDF76AFCE1780420FDF766FC44
:1033200010BD10B5044621780120FEF72FF8617812
:103330000220FEF72BF8A1780320FEF727F8E178AA
:103340000420FEF723F810BD10B5044621460020E6
:10335000FDF74CFC10BD10B5044621460020FEF7D9
:1033600015F810BD10B5044621461920FDF73EFCA6
:1033700010BD10B5044621461B20FEF707F810BD0E
:1033800010B5044621461720FDF77AFC10BD10B594
:10339000044621461920FEF731F810BD10B5044649
:1033A00021780F20FDF722FC61781020FDF71EFC2C
:1033B000A1781120FDF71AFCE1781220FDF716FC28
:1033C00010BD10B5044621780F20FDF7DFFF6178AE
:1033D0001020FDF7DBFFA1781120FDF7D7FFE17882
:1033E0001220FDF7D3FF10BD10B50446217805204B
:1033F000FDF7FCFB61780620FDF7F8FBA1780720BC
:10340000FDF7F4FBE1780820FDF7F0FB10BD10B5E7
:10341000044621780520FDF7B9FF61780620FDF705
:10342000B5FFA1780720FDF7B1FFE1780820FDF78F
:10343000ADFF10BD10B5002414E04FF4804101EB46
:1034400004211F318AB202211046FDF7CFFB4FF451
:10345000804101EB04211E318AB202211046FDF7A2
:10346000C5FB641C082CE8DB10BD704770B5034633
:103470000C4600214FF48040264D28805818000A41
:10348000254D287300BF2448007A00F00100002871
:10349000F9D02148007B58181F4D287300BF1E48E3
:1034A000007A00F001000028F9D01B48007BC2F32D
:1034B0000620194D287300BF1748007A00F001005C
:1034C0000028F9D01448007B134D2A7300BF12481E
:1034D000007A00F001000028F9D00F48007B00219D
:1034E0000EE000200C4D287300BF0B48007A00F05E
:1034F00001000028F9D0084D287B6054481C81B297
:103500009142EEDB4FF48045024EB61E35801046E8
:1035100070BD00001A0C02400030014070B5034637
:103520000C4600210AB9002070BD4FF48040274DA1
:1035300028805818000A264D287300BF2448007AB6
:1035400000F001000028F9D02148007B5818204DD8
:10355000287300BF1E48007A00F001000028F9D04F
:103560001B48007BC2F3062040F08000184D2873F2
:1035700000BF1748007A00F001000028F9D0144875
:10358000007B134D2A7300BF1148007A00F0010040
:103590000028F9D00E48007B00210DE0605C0C4D46
:1035A000287300BF0A48007A00F001000028F9D013
:1035B0000748007B481C81B29142EFDB4FF4804505
:1035C000024EB61E35801046AEE700001A0C0240CF
:1035D000003001402DE9F0478246884691461C465E
:1035E000C9F30A075046FEF7F1FAC5193819B0F5C4
:1035F000006F16DDC7F500618EB2ABB232464146B0
:103600001846FFF78BFFB044A11B8EB25046FEF761
:10361000DDFA05462B46324641461846FFF77EFF47
:1036200005E0ABB2224641461846FFF777FFBDE8FA
:10363000F087000053494E44303A31312E30322E5B
:10364000323031362020383A3435003C21444F4363
:10365000545950452068746D6C3E0D0A3C68746D79
:103660006C3E0D0A3C686561643E0D0A3C6D6574F4
:103670006120636861727365743D225554462D382C
:1036800022202F3E0D0A3C7469746C653ED09ED09A
:10369000B1D0BDD0BED0B2D0BBD0B5D0BDD0B8D0E7
:1036A000B520D0BFD180D0BED0B3D180D0B0D0BCF7
:1036B000D0BCD18B20D0BAD0BED0BDD182D180D0E9
:1036C000BED0BBD0BBD0B5D180D0B03C2F74697414
:1036D0006C653E0D0A3C7374796C653E0D0A626F31
:1036E0006479207B20666F6E742D73697A653A2049
:1036F00031656D3B20666F6E742D66616D696C7906
:103700003A20417269616C2C2048656C7665746959
:1037100063612C2073616E732D73657269663B2043
:10372000636F6C6F723A20233232323B206D6172CC
:1037300067696E3A2031656D3B207D0D0A646976BC
:10374000207B206D617267696E3A2031656D203093
:103750003B206C696E652D6865696768743A203135
:103760003530253B207D0D0A6831207B206D61724C
:1037700067696E3A203020302031656D3B20666FDE
:103780006E742D73697A653A20323030253B20669D
:103790006F6E742D7765696768743A206E6F726D0D
:1037A000616C3B207D0D0A6832207B206D61726761
:1037B000696E3A2032656D20302031656D3B2066A0
:1037C0006F6E742D73697A653A20313530253B2050
:1037D000666F6E742D7765696768743A206E6F72D4
:1037E0006D616C3B207D0D0A696E707574207B20C5
:1037F0006D617267696E3A20302032656D3B2070D2
:10380000616464696E673A20357078203130707871
:103810003B20626F726465723A2031707820736F5A
:103820006C696420236262623B207D0D0A696E70C0
:1038300075743A666F637573207B20626F7264657E
:10384000722D636F6C6F723A233239383062393BB4
:10385000207D0D0A627574746F6E207B206469731D
:10386000706C61793A20696E6C696E653B20706F8F
:10387000736974696F6E3A2072656C6174697665FC
:103880003B206F766572666C6F773A207669736954
:10389000626C653B2070616464696E673A203670C3
:1038A0007820313270783B20626F726465723A2002
:1038B0006E6F6E653B206261636B67726F756E64DD
:1038C0003A20233334393864623B20636F6C6F7263
:1038D0003A20236666663B206F75746C696E653AA4
:1038E000206E6F6E653B207D0D0A627574746F6E7D
:1038F0003A686F766572207B206261636B67726FD6
:10390000756E643A20233532613765303B2063752C
:1039100072736F723A706F696E7465723B207D0DC1
:103920000A627574746F6E3A616374697665207BA0
:1039300020746F703A203170783B206C6566743A61
:10394000203170783B206261636B67726F756E64C3
:103950003A20233233383663383B207D0D0A6275B6
:1039600074746F6E3A3A2D6D6F7A2D666F6375734E
:103970002D696E6E6572207B20626F726465723A8B
:1039800020303B207D0D0A61207B20636F6C6F72BD
:103990003A20233232323B20746578742D6465639B
:1039A0006F726174696F6E3A206E6F6E653B207D39
:1039B0000D0A23666163746F72792D6461746120EE
:1039C0007B20646973706C61793A206E6F6E653B21
:1039D000207D0D0A23666163746F72792D646174B2
:1039E00061206C6162656C207B20646973706C611E
:1039F000793A20696E6C696E652D626C6F636B3B02
:103A00002077696474683A20383070783B207D0DE7
:103A10000A23666163746F72792D64617461206931
:103A20006E707574207B2077696474683A20333037
:103A30003070783B206D617267696E3A20302031BA
:103A4000656D203020303B207D0D0A237374617436
:103A50007573207B20636F6C6F723A202366303061
:103A60003B20666F6E742D73697A653A203135306C
:103A7000253B20746578742D616C69676E3A20630C
:103A8000656E7465723B207D0D0A23696E737461E7
:103A90006C6C207B207669736962696C6974793A11
:103AA0002068696464656E3B207D0D0A3C2F737449
:103AB000796C653E0D0A3C2F686561643E0D0A3CD9
:103AC000626F64793E0D0A3C68313ED0A0D0B5D01B
:103AD000B6D0B8D0BC20D0BED0B1D0BDD0BED0B250
:103AE000D0BBD0B5D0BDD0B8D18F20D0BFD180D081
:103AF000BED0B3D180D0B0D0BCD0BCD18B20D0BA96
:103B0000D0BED0BDD182D180D0BED0BBD0BBD0B5CD
:103B1000D1803C6120687265663D226A617661737E
:103B200063726970743A766F69642830293B222089
:103B300069643D22666163746F72792D646174619A
:103B40002D73686F77223ED0B03C2F613E3C2F68CA
:103B5000313E0D0A3C6469763E3C627574746F6E4A
:103B600020747970653D22627574746F6E222069CD
:103B7000643D226578697422207469746C653D2205
:103B8000D092D18BD0B9D182D0B820D0B8D0B720C4
:103B9000D180D0B5D0B6D0B8D0BCD0B020D0BFD1B5
:103BA00080D0BED0B3D180D0B0D0BCD0BCD0B8D142
:103BB00080D0BED0B2D0B0D0BDD0B8D18F223ED050
:103BC00092D18BD0B9D182D0B820D0B8D0B720D183
:103BD00080D0B5D0B6D0B8D0BCD0B020D0BED0B197
:103BE000D0BDD0BED0B2D0BBD0B5D0BDD0B8D18FB3
:103BF00020D0BFD180D0BED0B3D180D0B0D0BCD087
:103C0000BCD18B3C2F627574746F6E3E3C2F64691F
:103C1000763E0D0A3C6469762069643D22666163E4
:103C2000746F72792D64617461223E0D0A3C6832B2
:103C30003ED0A3D181D182D0B0D0BDD0BED0B2D041
:103C4000BAD0B020D0B7D0B0D0B2D0BED0B4D1812D
:103C5000D0BAD0B8D18520D0B4D0B0D0BDD0BDD1ED
:103C60008BD1853C2F68323E0D0A3C6469763E3C20
:103C70006C6162656C20666F723D22666163746F71
:103C800072792D646174612D7077223ED09FD0B01F
:103C9000D180D0BED0BBD18C3A3C2F6C6162656CB8
:103CA0003E3C696E70757420747970653D22746550
:103CB0007874222069643D22666163746F72792D85
:103CC000646174612D707722202F3E3C2F646976E9
:103CD0003E0D0A3C6469763E3C6C6162656C206610
:103CE0006F723D22666163746F72792D64617461D5
:103CF0002D736572223ED0A1D0B5D1802FD0BD3AB0
:103D00003C2F6C6162656C3E3C696E70757420740A
:103D10007970653D2274657874222069643D22665D
:103D20006163746F72792D646174612D73657222A1
:103D3000202F3E3C627574746F6E20747970653DFF
:103D400022627574746F6E222069643D226661631D
:103D5000746F72792D646174612D7365722D696E53
:103D600063223E2B3C2F627574746F6E3E3C2F6451
:103D700069763E0D0A3C6469763E3C6C6162656C16
:103D800020666F723D22666163746F72792D646183
:103D900074612D737472223ED0A1D182D180D0BEC5
:103DA000D0BAD0B03A3C2F6C6162656C3E3C696E13
:103DB00070757420747970653D2274657874222062
:103DC00069643D22666163746F72792D6461746108
:103DD0002D73747222202F3E3C2F6469763E0D0AAB
:103DE0003C6469763E3C6C6162656C20666F723D36
:103DF00022666163746F72792D646174612D7365DD
:103E00006E64223E3C2F6C6162656C3E3C62757450
:103E1000746F6E20747970653D22627574746F6E74
:103E2000222069643D22666163746F72792D64613A
:103E300074612D73656E64223ED0A3D181D182D08E
:103E4000B0D0BDD0BED0B2D0B8D182D18C3C2F6220
:103E50007574746F6E3E3C2F6469763E0D0A3C2F7C
:103E60006469763E0D0A3C68323ED092D0BED18164
:103E7000D181D182D0B0D0BDD0BED0B2D0BBD0B570
:103E8000D0BDD0B8D0B520D0BAD0BED0BDD182D1AF
:103E900080D0BED0BBD0BBD0B5D180D0B03C2F68D5
:103EA000323E0D0A3C6469763E3C627574746F6EF6
:103EB00020747970653D22627574746F6E2220697A
:103EC000643D22636C6561722D63616C63222074B2
:103ED00069746C653D22D0A3D0B4D0B0D0BBD0B84B
:103EE000D182D18C20D0BFD180D0BED0B3D180D0F0
:103EF000B0D0BCD0BCD18320D0B4D0BED180D0B0A3
:103F0000D181D187D0B5D182D0B0223ED0A3D0B458
:103F1000D0B0D0BBD0B8D182D18C20D0BFD180D08E
:103F2000BED0B3D180D0B0D0BCD0BCD18320D0B46F
:103F3000D0BED180D0B0D181D187D0B5D182D0B020
:103F40003C2F627574746F6E3E0D0A3C627574741A
:103F50006F6E20747970653D22627574746F6E2285
:103F60002069643D22636C6561722D636F6E6669C2
:103F70006722207469746C653D22D0A3D0B4D0B0A0
:103F8000D0BBD0B8D182D18C20D0BAD0BED0BDD1D8
:103F900084D0B8D0B3D183D180D0B0D186D0B8D1BD
:103FA0008E223ED0A3D0B4D0B0D0BBD0B8D182D175
:103FB0008C20D0BAD0BED0BDD184D0B8D0B3D183FC
:103FC000D180D0B0D186D0B8D18E3C2F62757474B8
:103FD0006F6E3E3C2F6469763E0D0A3C68323ED0DF
:103FE0009ED0B1D0BDD0BED0B2D0BBD0B5D0BDD0A8
:103FF000B8D0B520D184D0B0D0B9D0BBD0B020D00B
:10400000BFD180D0BED0B3D180D0B0D0BCD0BCD1D5
:104010008B3C2F68323E0D0A3C6469763ED092D1CB
:104020008BD0B1D0B5D180D0B8D182D0B520D184D9
:10403000D0B0D0B9D0BB20D0BFD180D0BED0B3D10A
:1040400080D0B0D0BCD0BCD18B3A3C696E70757456
:1040500020747970653D2266696C65222069643D33
:104060002266696C6522206175746F636F6D706C78
:104070006574653D226F666622202F3E3C2F646981
:10408000763E0D0A3C6469762069643D2266696C5F
:10409000652D696E666F223E3C2F6469763E0D0A7F
:1040A0003C6469763E3C627574746F6E20747970FE
:1040B000653D22627574746F6E222069643D2269C9
:1040C0006E7374616C6C22207469746C653D22D0CF
:1040D000A3D181D182D0B0D0BDD0BED0B2D0B8D122
:1040E00082D18C20D0B2D18BD0B1D180D0B0D0BD14
:1040F000D0BDD183D18E20D0BFD180D0BED0B3D19E
:1041000080D0B0D0BCD0BCD183223ED0A3D181D14D
:1041100082D0B0D0BDD0BED0B2D0B8D182D18C20A8
:10412000D0B2D18BD0B1D180D0B0D0BDD0BDD183F1
:10413000D18E20D0BFD180D0BED0B3D180D0B0D06E
:10414000BCD0BCD1833C2F627574746F6E3E3C2F23
:104150006469763E0D0A3C6469762069643D227389
:104160007461747573223E3C2F6469763E0D0A3C7F
:104170007363726970743E0D0A76617220643D2229
:104180003139322E3136382E312E32222C653D22F5
:104190002C222C663D22223B66756E6374696F6E1D
:1041A00020672861297B72657475726E2031303EFC
:1041B000613F2230222B613A22222B617D66756E8F
:1041C0006374696F6E206928297B666F7228766137
:1041D0007220613D5B66756E6374696F6E28297B22
:1041E00072657475726E206E657720584D4C4874F8
:1041F0007470526571756573747D2C66756E637429
:10420000696F6E28297B72657475726E206E657792
:1042100020416374697665584F626A656374282229
:104220004D73786D6C322E584D4C485454502229A1
:104230007D2C66756E6374696F6E28297B72657458
:1042400075726E206E657720416374697665584F8C
:10425000626A65637428224D73786D6C332E584DF5
:104260004C4854545022297D2C66756E6374696FD6
:104270006E28297B72657475726E206E6577204199
:104280006374697665584F626A65637428224D6964
:1042900063726F736F66742E584D4C48545450229D
:1042A000297D5D2C633D21312C623D303B623C61B8
:1042B0002E6C656E6774683B622B2B297B74727958
:1042C0007B633D615B625D28297D6361746368285F
:1042D0006E297B636F6E74696E75657D6272656150
:1042E0006B7D72657475726E20637D66756E637426
:1042F000696F6E206A28612C632C62297B612E61B4
:1043000064644576656E744C697374656E65723F5E
:10431000612E6164644576656E744C697374656E74
:10432000657228632C622C2131293A612E617474E4
:104330006163684576656E743F612E617474616374
:10434000684576656E7428226F6E222B632C622975
:104350003A615B226F6E222B635D3D627D0A66755A
:104360006E6374696F6E206D2861297B7265747548
:10437000726E20646F63756D656E742E676574452B
:104380006C656D656E74427949642861297D667536
:104390006E6374696F6E206F28612C63297B766170
:1043A0007220623D612B322A633B623D652E636859
:1043B000617241742862292B652E636861724174B1
:1043C00028622B31293B32213D622E6C656E677469
:1043D000683F623D6E756C6C3A28623D7061727325
:1043E00065496E7428622C3136292C623D69734E02
:1043F000614E2862293F6E756C6C3A62293B72658A
:104400007475726E20537472696E672E66726F6D6A
:1044100043686172436F64652862297D66756E63C7
:1044200074696F6E207028612C63297B766172201D
:10443000633D632B31322C623D7B747970653A6148
:104440002C643A7061727365496E74286F28632C0E
:1044500030292B6F28632C31292C3130292C6D3ACF
:104460007061727365496E74286F28632C33292B31
:104470006F28632C34292C3130292C793A706172E1
:104480007365496E74286F28632C36292B6F286357
:104490002C37292B6F28632C38292B6F28632C3954
:1044A000292C3130292C683A7061727365496E7419
:1044B000286F28632C3131292B6F28632C31322946
:1044C0002C3130292C693A7061727365496E7428F9
:1044D0006F28632C3134292B6F28632C3135292C1C
:1044E0003130297D3B72657475726E20622E74794D
:1044F00070652B223A222B6728622E64292B222EEC
:10450000222B6728622E6D292B222E222B672862F0
:104510002E79292B2220222B6728622E68292B2214
:104520003A222B6728622E69297D0A66756E6374AC
:10453000696F6E20712861297B6D282266696C6520
:104540002D696E666F22292E696E6E657248544D14
:104550004C3D617D66756E6374696F6E2072286173
:10456000297B6D282273746174757322292E696EFC
:104570006E657248544D4C3D612E7265706C61637E
:1045800065282F5C6E2F69672C223C6272202F3EBB
:1045900022297D66756E6374696F6E2073286129A8
:1045A0007B76617220633D742C623D6928293B62F1
:1045B0002E6F6E726561647973746174656368618E
:1045C0006E67653D66756E6374696F6E28297B340E
:1045D0003D3D622E7265616479537461746526266F
:1045E00028636C65617254696D656F7574286E29F6
:1045F0002C632626632829297D3B622E6F70656E09
:104600002822706F7374222C222F222C2130293BF8
:10461000622E736574526571756573744865616463
:1046200065722822436F6E74656E742D54797065BF
:10463000222C226170706C69636174696F6E2F78CF
:104640002D7777772D666F726D2D75726C656E6341
:104650006F64656422293B622E73656E642861294C
:104660003B722822D092D18BD0BFD0BED0BBD0BD60
:10467000D18FD0B5D182D181D18F20D0BED0BFD043
:10468000B5D180D0B0D186D0B8D18F2C20D0BFD0BA
:10469000BED0B6D0B0D0BBD183D0B9D181D182D079
:1046A000B02C20D0B6D0B4D0B8D182D0B52E2E2E1A
:1046B00022293B766172206E3D73657454696D6585
:1046C0006F75742866756E6374696F6E28297B62D6
:1046D0002E61626F727428293B722822D09AD0BE54
:1046E000D0BDD182D180D0BED0BBD0BBD0B5D1801F
:1046F00020D0BDD0B520D0BED182D0B2D0B5D18728
:10470000D0B0D0B5D18222297D2C334534297D0A01
:1047100066756E6374696F6E207528612C63297BE2
:1047200076617220623D6928293B622E6F6E726548
:1047300061647973746174656368616E67653D6611
:10474000756E6374696F6E28297B343D3D622E72ED
:10475000656164795374617465262628636C6561AC
:104760007254696D656F7574286E292C63262663F3
:104770002829297D3B622E6F70656E28226765743B
:10478000222C222F3F222B612C2130293B622E73B9
:10479000656E6428293B722822D092D18BD0BFD07D
:1047A000BED0BBD0BDD18FD0B5D182D181D18F2029
:1047B000D0BED0BFD0B5D180D0B0D186D0B8D18F47
:1047C0002C20D0BFD0BED0B6D0B0D0BBD183D0B912
:1047D000D181D182D0B02C20D0B6D0B4D0B8D18283
:1047E000D0B52E2E2E22293B766172206E3D736548
:1047F0007454696D656F75742866756E6374696F3E
:104800006E28297B622E61626F727428293B7228A0
:1048100022D09AD0BED0BDD182D180D0BED0BBD064
:10482000BBD0B5D18020D0BDD0B520D0BED182D0F4
:10483000B2D0B5D187D0B0D0B5D18222297D2C316C
:104840004534297D66756E6374696F6E20742829FE
:104850007B722822D09ED0BFD0B5D180D0B0D18677
:10486000D0B8D18F20D0B2D18BD0BFD0BED0BBD0EA
:10487000BDD0B5D0BDD0B05C6ED094D0B0D0BDD0DE
:10488000BDD0B0D18F20D181D182D180D0B0D0BD68
:10489000D0B8D186D0B020D0BED0B1D0BDD0BED09F
:1048A000B2D0B8D182D181D18F20D187D0B5D1807B
:1048B000D0B5D0B7203520D181D0B5D0BAD183D0F2
:1048C000BDD0B422293B73657454696D656F7574EE
:1048D0002866756E6374696F6E28297B77696E64CC
:1048E0006F772E6C6F636174696F6E2E72656C6F7B
:1048F000616428297D2C354533297D0A66756E63F0
:1049000074696F6E207628297B722822D09ED0BFD2
:10491000D0B5D180D0B0D186D0B8D18F20D0B2D18F
:104920008BD0BFD0BED0BBD0BDD0B5D0BDD0B05CD9
:104930006ED09FD0B5D180D0B5D0BDD0B0D0BFD1D2
:1049400080D0B0D0B2D0BBD0B5D0BDD0B8D0B5201B
:10495000D0BDD0B020D0B1D0B0D0B7D0BED0B2D1C1
:104960008BD0B920D0B0D0B4D180D0B5D18120D0F7
:10497000BAD0BED0BDD182D180D0BED0BBD0BBD04A
:10498000B5D180D0B02028222B642B222920D187BA
:10499000D0B5D180D0B5D0B7203520D181D0B5D019
:1049A000BAD183D0BDD0B422293B73657454696DEC
:1049B000656F75742866756E6374696F6E28297BE0
:1049C00077696E646F772E6C6F636174696F6E3D8B
:1049D00022687474703A2F2F222B642B222F227D91
:1049E0002C354533297D66756E6374696F6E20774B
:1049F00028297B722822D09ED0BFD0B5D180D0B0DC
:104A0000D186D0B8D18F20D0B2D18BD0BFD0BED07C
:104A1000BBD0BDD0B5D0BDD0B022297D0A696628F3
:104A20002177696E646F772E46696C657C7C21778F
:104A3000696E646F772E46696C6552656164657254
:104A40007C7C2177696E646F772E46696C654C6952
:104A5000737429722822D092D0B0D18820D0B1D1DD
:104A600080D0B0D183D0B7D0B5D18020D0BDD0B563
:104A700020D0BFD0BED0B4D0B4D0B5D180D0B6D0C5
:104A8000B8D0B2D0B0D0B5D18220D0BCD0B5D1850D
:104A9000D0B0D0BDD0B8D0B7D0BC20D0BFD0B5D169
:104AA00080D0B5D0BFD180D0BED0B3D180D0B0D06F
:104AB000BCD0BCD0B8D180D0BED0B2D0B0D0BDD0E8
:104AC000B8D18F20D0BAD0BED0BDD182D180D0BED7
:104AD000D0BBD0BBD0B5D180D0B02E5C6E5C6ED0D8
:104AE00092D0BED181D0BFD0BED0BBD18CD0B7D1F7
:104AF00083D0B9D182D0B5D181D18C20D0BED0B4F1
:104B0000D0BDD0B8D0BC20D0B8D0B720D181D0BBD8
:104B1000D0B5D0B4D183D18ED189D0B8D18520D0B1
:104B2000B1D180D0B0D183D0B7D0B5D180D0BED0F4
:104B3000B23A5C6E496E7465726E65742045787029
:104B40006C6F7265722031302E3020D0B820D0B218
:104B5000D18BD188D0B52C5C6E4D6F7A696C6C614D
:104B60002046697265666F7820332E3620D0B820D3
:104B7000D0B2D18BD188D0B52C5C6E476F6F676C8B
:104B800065204368726F6D6520372E3020D0B820C5
:104B9000D0B2D18BD188D0B52C5C6E4F706572616C
:104BA0002031312E353020D0B820D0B2D18BD188F1
:104BB000D0B52E22292C6D282266696C6522292EFB
:104BC00064697361626C65643D21303B0A6A286DDB
:104BD000282266696C6522292C226368616E6765EC
:104BE000222C66756E6374696F6E28297B766172FC
:104BF00020613D6D282266696C6522292E66696CEC
:104C000065735B305D3B69662861297B7661722044
:104C1000633D27D092D18BD0B1D180D0B0D0BD2010
:104C2000D184D0B0D0B9D0BB203C656D3E22272BBB
:104C3000612E6E616D652B27223C2F656D3E2C2009
:104C4000272B28612E73697A652F31303234292E53
:104C5000746F466978656428292B2220D0BAD0B1B8
:104C60002E222C623D6E65772046696C6552656127
:104C70006465723B622E7265616441735465787439
:104C80002861293B622E6F6E6C6F61643D66756EA4
:104C90006374696F6E2862297B666F722876617211
:104CA00020623D622E7461726765742E7265737541
:104CB0006C742E73706C697428223A303230303044
:104CC00030303422292C613D5B5D2C783D312C6BDA
:104CD0003B6B3D625B782B2B5D3B297B76617220C1
:104CE0006C3D6B2E737562737472696E6728302C1D
:104CF00034292C683D7061727365496E74286C2C80
:104D00003130293B69662821283830303E687C7C68
:104D10003930303C6829297B6B3D6B2E73706C6990
:104D20007428225C6E22293B303D3D612E6C656EFD
:104D30006774682626612E7075736828223A222BC4
:104D40006C293B666F72286C3D323B683D6B5B6C37
:104D50002B2B5D3B29683D682E736C696365283990
:104D60002C2D33292C612E707573682868292C30FE
:104D70003D3D286C2637292626612E7075736828DC
:104D8000222122297D7D663D612E6A6F696E28226F
:104D900022293B653D662E73706C6974282221229E
:104DA000292E6A6F696E282222293B623D652E6991
:104DB0006E6465784F66282235333439344534348F
:104DC0003330334122293B613D652E696E6465783D
:104DD0004F6628223533343934453434353733413E
:104DE00022293B0A303E627C7C303E613F2871289C
:104DF000632B223C6272202F3E3C7374726F6E678D
:104E00003ED09DD0B5D0BAD0BED180D180D0B5D063
:104E1000BAD182D0BDD18BD0B920D184D0B0D0B995
:104E2000D0BB20D0BFD180D0BED0B3D180D0B0D045
:104E3000BCD0BCD18B213C2F7374726F6E673E2245
:104E4000292C6D2822696E7374616C6C22292E7373
:104E500074796C652E7669736962696C6974793DE1
:104E60002268696464656E22293A287128632B22BE
:104E70003C6272202F3ED09AD0BED180D180D0B576
:104E8000D0BAD182D0BDD18BD0B920D184D0B0D00E
:104E9000B9D0BB20D0BFD180D0BED0B3D180D0B0EC
:104EA000D0BCD0BCD18B213C6272202F3E3C6272C0
:104EB000202F3ED092D0B5D180D181D0B8D18F20D3
:104EC000D0BFD180D0BED0B3D180D0B0D0BCD0BC08
:104ED000D18B20D0BAD0BED0BDD182D180D0BED0AF
:104EE000BBD0BBD0B5D180D0B03A203C7374726FC8
:104EF0006E673E222B70282253494E30222C6229A5
:104F00002B223C2F7374726F6E673E2C3C627220B2
:104F10002F3ED092D0B5D180D181D0B8D18F20D0C2
:104F2000BFD180D0BED0B3D180D0B0D0BCD0BCD1A6
:104F30008B20D0BAD0BED0BDD184D0B8D0B3D1836D
:104F4000D180D0B0D182D0BED180D0B03A203C73D5
:104F500074726F6E673E222B70282253494E57227F
:104F60002C61292B223C2F7374726F6E673E2E22A8
:104F7000292C6D2822696E7374616C6C22292E7342
:104F800074796C652E7669736962696C6974793DB0
:104F90002276697369626C6522297D7D656C736513
:104FA0002071282222297D293B6A286D28226661EA
:104FB00063746F72792D646174612D73686F7722E9
:104FC000292C22636C69636B222C66756E6374698D
:104FD0006F6E28297B6D2822666163746F72792D4C
:104FE0006461746122292E7374796C652E6469730F
:104FF000706C61793D22626C6F636B227D293B0A84
:105000006A286D2822666163746F72792D646174F9
:10501000612D7365722D696E6322292C22636C6980
:10502000636B222C66756E6374696F6E28297B76BC
:10503000617220613D6D2822666163746F72792D03
:10504000646174612D73657222293B612E76616CF7
:1050500075653D7061727365496E7428612E766165
:105060006C75652C3130292B313B612E666F637571
:105070007328297D293B6A286D2822666163746F35
:1050800072792D646174612D73656E6422292C22FE
:10509000636C69636B222C66756E6374696F6E282E
:1050A000297B76617220613D6D2822666163746F91
:1050B00072792D646174612D707722292E76616C6E
:1050C00075652C633D6D2822666163746F72792D5E
:1050D000646174612D73657222292E76616C756529
:1050E0002C623D6D2822666163746F72792D646154
:1050F00074612D73747222292E76616C75653B691B
:10510000662821617C7C21637C7C216229616C653D
:1051100072742822D094D0BED0BBD0B6D0BDD18B73
:1051200020D0B1D18BD182D18C20D0B7D0B0D0BF1C
:10513000D0BED0BBD0BDD0B5D0BDD18B20D0B2D1E8
:1051400081D0B520D0BFD0BED0BBD18F2C20D0BE57
:10515000D0BFD0B5D180D0B0D186D0B8D18F20D03B
:10516000BED182D0BCD0B5D0BDD0B5D0BDD0B022DC
:10517000293B656C73657B666F72283B363E632EF8
:105180006C656E6774683B29633D2230222B633B5C
:10519000636F6E6669726D2822D09FD0BED0B4D185
:1051A00082D0B2D0B5D180D0B4D0B8D182D0B52021
:1051B000D183D181D182D0B0D0BDD0BED0B2D0BA4F
:1051C000D18320D0B7D0B0D0B2D0BED0B4D181D0AE
:1051D000BAD0B8D18520D0B4D0B0D0BDD0BDD18B9D
:1051E000D18522293F752822536574503D7B222B9F
:1051F000612B223A53222B632B622B227D222C77A8
:10520000293A616C6572742822D09ED0BFD0B5D186
:1052100080D0B0D186D0B8D18F20D0BED182D0BCC2
:10522000D0B5D0BDD0B5D0BDD0B022297D7D293B31
:105230000A6A286D2822696E7374616C6C22292CAD
:1052400022636C69636B222C66756E6374696F6E82
:1052500028297B216D282266696C6522292E6669C2
:105260006C65735B305D7C7C21663F722822D0A325
:10527000D0BAD0B0D0B6D0B8D182D0B520D0BAD0C4
:10528000BED180D180D0B5D0BAD182D0BDD18BD0A3
:10529000B920D184D0B0D0B9D0BB20D0BFD180D07C
:1052A000BED0B3D180D0B0D0BCD0BCD18B22293AF3
:1052B0007328224669726D4845583D7B222B662B28
:1052C000227D22297D293B6A286D2822636C656135
:1052D000722D63616C6322292C22636C69636B22DB
:1052E0002C66756E6374696F6E28297B76617220F7
:1052F000613D70726F6D70742827D092D0BDD0B8A8
:10530000D0BCD0B0D0BDD0B8D0B52120D09FD180F6
:10531000D0BED0B3D180D0B0D0BCD0BCD0B020D023
:10532000B4D0BED180D0B0D181D187D0B5D182D018
:10533000B020D0B1D183D0B4D0B5D18220D183D028
:10534000B4D0B0D0BBD0B5D0BDD0B020D0B1D0B5E6
:10535000D0B720D0B2D0BED0B7D0BCD0BED0B6D09F
:10536000BDD0BED181D182D0B820D0B2D0BED18143
:10537000D181D182D0B0D0BDD0BED0B2D0BBD0B55B
:10538000D0BDD0B8D18F5C6ED094D0BBD18F20D09F
:10539000BFD0BED182D0B2D0B5D180D0B6D0B4D03B
:1053A000B5D0BDD0B8D18F20D0B2D0B2D0B5D0B4A6
:1053B000D0B8D182D0B520D0B220D0BFD0BED0BB23
:1053C000D0B520D181D0BBD0BED0B2D0BE2022D0AB
:1053D000A3D094D090D09BD098D0A2D0AC22272933
:1053E0003B61262622D183D0B4D0B0D0BBD0B8D177
:1053F00082D18C223D3D612E746F4C6F7765724374
:1054000061736528293F752822436C656172436189
:105410006C63222C77293A616C6572742822D09EC5
:10542000D0BFD0B5D180D0B0D186D0B8D18F20D068
:10543000BED182D0BCD0B5D0BDD0B5D0BDD0B02209
:10544000297D293B0A6A286D2822636C6561722DCB
:10545000636F6E66696722292C22636C69636B2215
:105460002C66756E6374696F6E28297B7661722075
:10547000613D70726F6D70742822D092D0BDD0B82B
:10548000D0BCD0B0D0BDD0B8D0B52120D09AD0BE3D
:10549000D0BDD184D0B8D0B3D183D180D0B0D186A3
:1054A000D0B8D18F20D0BAD0BED0BDD182D180D0DB
:1054B000BED0BBD0BBD0B5D180D0B020D0B1D183CD
:1054C000D0B4D0B5D18220D183D0B4D0B0D0BBD0AD
:1054D000B5D0BDD0B020D0B1D0B5D0B720D0B2D0EB
:1054E000BED0B7D0BCD0BED0B6D0BDD0BED181D199
:1054F00082D0B820D0B2D0BED181D181D182D0B0FB
:10550000D0BDD0BED0B2D0BBD0B5D0BDD0B8D18F79
:105510005C6E49502DD0B0D0B4D180D0B5D18120AF
:10552000D0BAD0BED0BDD182D180D0BED0BBD0BB8E
:10553000D0B5D180D0B020D0B1D183D0B4D0B5D146
:105540008220D183D181D182D0B0D0BDD0BED0B2A3
:10555000D0BBD0B5D0BD20D0BFD0BE20D183D0BC71
:10556000D0BED0BBD187D0B0D0BDD0B8D18E202D89
:1055700020222B642B275C6ED094D0BBD18F20D0FF
:10558000BFD0BED182D0B2D0B5D180D0B6D0B4D049
:10559000B5D0BDD0B8D18F20D0B2D0B2D0B5D0B4B4
:1055A000D0B8D182D0B520D0B220D0BFD0BED0BB31
:1055B000D0B520D181D0BBD0BED0B2D0BE2022D0B9
:1055C000A3D094D090D09BD098D0A2D0AC22272941
:1055D0003B61262622D183D0B4D0B0D0BBD0B8D185
:1055E00082D18C223D3D612E746F4C6F7765724382
:1055F00061736528293F752822436C656172436F8A
:105600006E66222C76293A616C6572742822D09ECF
:10561000D0BFD0B5D180D0B0D186D0B8D18F20D076
:10562000BED182D0BCD0B5D0BDD0B5D0BDD0B02217
:10563000297D293B6A286D28226578697422292CE6
:1056400022636C69636B222C66756E6374696F6E7E
:1056500028297B636F6E6669726D2822D09FD0BE49
:10566000D0B4D182D0B2D0B5D180D0B4D0B8D182AC
:10567000D0B520D0B2D18BD185D0BED0B420D0B897
:10568000D0B720D180D0B5D0B6D0B8D0BCD0B02063
:10569000D0BED0B1D0BDD0BED0B2D0BBD0B5D0BDC1
:1056A000D0B8D18F20D0BFD180D0BED0B3D180D0E0
:1056B000B0D0BCD0BCD18B20D0BAD0BED0BDD182AE
:1056C000D180D0BED0BBD0BBD0B5D180D0B0222944
:1056D0003F73282272756E6D61696E3D7B317D224C
:1056E000293A616C6572742822D09ED0BFD0B5D1A2
:1056F00080D0B0D186D0B8D18F20D0BED182D0BCDE
:10570000D0B5D0BDD0B5D0BDD0B022297D293B0ABF
:105710003C2F7363726970743E0D0A3C2F626F6494
:10572000793E0D0A3C2F68746D6C3E00648A1788C0
:105730004B360008000000002B5700080040404096
:105740004040404040404141414141404040404054
:105750004040404040404040404040404005020200
:1057600002020202020202020202020202202020BF
:10577000202020202020200202020202020290901B
:105780009090909010101010101010101010101019
:10579000101010101010101002020202020288886D
:1057A0008888888808080808080808080808080879
:1057B0000808080808080808020202024000000061
:1057C0003D570008485454502F312E31203230308C
:1057D000204F4B200D0A436F6E6E656374696F6EC8
:1057E0003A20636C6F73650D0A4163636573732DB3
:1057F000436F6E74726F6C2D416C6C6F772D4F72AE
:105800006967696E3A2A0D0A0D0A2052656164794A
:10581000210D0A0D0A000000485454502F312E313A
:1058200020323030204F4B200D0A436F6E6E65637F
:1058300074696F6E3A20636C6F73650D0A41636320
:105840006573732D436F6E74726F6C2D416C6C6F4A
:10585000772D4F726967696E3A2A0D0A0D0A0000AA
:105860008058000800000020400200003E030008AD
:105870001C59000840020020308E0000C81A0008A1
:1058800011847A030A0009ED0102030406070809DE
:10589000123512011B4003052A41052A42052A43FD
:1058A000052A44052A45052A46052A4705134020AE
:1058B00082089A410C9A420C9A430C9A440C9A45DD
:1058C0000C9A460C9A470C111209022C02232E0145
:1058D0001B0309041A29041A49041A69041A8904C1
:1058E0001AA9041AC90422E933200A2A26052B2002
:1058F0002A0A29052B204A0A29052B206A0A29058C
:105900002B208A0A29052B20AA0A29052B20CA0A3E
:0C59100029052B20EA0A2905CA09A2007B
:020000044002B8
:1040000001FF01FF01FF01FF01FF01FF01FF01FFB0
:0C40100001FF01FF01FF01FF012400007F
:040000050800018965
:00000001FF
